:020000020000FC
:10000000B3CDAEC10000000020C000008EC00000D3
:10001000000098C000000000000000000203040679
:10002000080C10182030406080000406080C1018DE
:100030002030406080A0C0000003070F1F000D0D9E
:1000400004050D050305030302004FB662FD0CC055
:10005000552041F00994C52DC095089483FDC7959E
:10006000C4BD64604FBE1895C0916400089483FDC0
:10007000C795C4BD6B7FC0916400CF3F09F41EC01B
:1000800070FF1AC082FD05C04FBE9198909893985A
:10009000189576FD0EC065FD0CC0C091B100C0FD85
:1000A0009498C1FD9798C2FD9598CAEFC095CA95DE
:1000B000F1F79198909893984FBE189524BCCC274F
:1000C000C064C8BF6460F8CFC6CF70FFC4CF65FD01
:1000D000C2CF919AC0CF70FFBECF65FDBCCF909AC2
:1000E000BACF70FFB8CF65FDB6CF939AB4CF949ACC
:1000F00070FFB1CF65FDAFCFC7E0CA95F1F7919A18
:10010000AACF979A70FFA7CF65FDA5CFC7E0CA9584
:10011000F1F7909AA0CF959A70FF9DCF65FD9BCF88
:10012000C7E0CA95F1F7939A96CF4FB6C9B7CF7E7D
:10013000C9BF6E7FCCB5CE0DDDB5DF1DDBBDCABD41
:100140004FBE18953FB68F7EABB7A074A2118061E9
:10015000A0E0ABBFA9B7AE7FA9BF7894A09168001B
:10016000AA2341F085FD2AC0A0916800AA95A0931A
:10017000680024C040E050E085FD14C0A0B396FFA5
:10018000A095A2FD4FEFA3E096FFA2E0A5BFAA278E
:10019000A064AABF8D7FA0B396FFA095A2FD5FEFDC
:1001A000451741F7A8E161FDA093680085FD03C0F4
:1001B000A8E1A093680040939600816085FD0EC081
:1001C000A0916900AA2331F0A0916900AA95A0939B
:1001D000690004C08061AA27A064AABF80FF3CC058
:1001E000A09196004A2F61FF8E7F85FD1CC0A091D3
:1001F000B400A430C1F4403F08F040EFA42FA29512
:10020000AF704A0F5091B600533069F0A695A6958D
:1002100050FD01C0A69552FD03C0A41B4A2F03C088
:100220004A0F08F44FEF40936100A72FA670A1F08A
:1002300073FD12C0A0917000AA0FAA0F50919E00EA
:1002400056955695541708F0452F4A0F4093610074
:1002500018F4AFEFA09361004091B400443009F06E
:100260003EC0A0916100A093630040916300A09103
:100270009B004A1708F04A2FA0919D004A1708F0EA
:100280004A2F542EA091A000AA2309F422C0542F73
:100290005A1B10F4A42F50E0BA2E8894AA1FAA2E3D
:1002A000A091A200A095AA22A50E58F0A091A100AD
:1002B000A21509F0AA95AA0EA093A10048F04A2D14
:1002C00008C0A091A100BA1608F0A395A093A100C0
:1002D0004FEF409364007F7B485F08F07064A52D6A
:1002E000A03408F06860A0916000A395A09360001E
:1002F00051F0F894A9B7A160A9BF84FF02C0A0E49F
:10030000ABBF3FBE1895A0917400A395A093740055
:1003100041E050916800552329F085FF03C05A95AC
:1003200050936800A0919600A13018F02092990097
:100330000DC020929A002092A300A0919900AF5F77
:10034000A093990018F0AFEFA0939900F894A9B783
:10035000A160A9BF84FF02C0A0E4ABBF3FBE189557
:100360003FB64CB55DB58F7EABB7A074A21180616E
:10037000A0E0ABBFA9B7AE7FA9BF789481FD23C031
:10038000A2E096FFA3E0A5BF8260A0B396FFA09570
:10039000A2FF05C040936500509366003EC1A3E0F4
:1003A00096FFA2E0A5BFAA27A064AABF8D7F85FF04
:1003B00001C026C140E0A0B396FFA095A2FD20C1D8
:1003C000409396000FC1A3E096FFA2E0A5BF8D7FEA
:1003D00061FF71C0A2E096FFA3E0A5BFAA27A064B9
:1003E000AABF82604093910050939200A0908F002A
:1003F0004A19B09090005B09BB24A22C4C385205DE
:1004000018F42092950049C0A091D400AA2359F174
:10041000483C520528F4A0E1BA2EAAE0AA2E23C037
:100420004836A1E05A0728F4A8E0BA2EAFE0AA2E79
:100430001AC0403DA2E05A0728F4A4E0BA2EAEE16B
:10044000AA2E11C0403AA5E05A0728F4A2E0BA2E1D
:10045000ACE3AA2E08C04839A8E05A0720F4A1E06E
:10046000BA2EA8E7AA2EC42EA0919300CA1AD52EA0
:10047000A0919400DA0ADD202AF4AFEFC094D09462
:10048000CA1ADA0A20929500A8E0A210A0E0CA14C5
:10049000DA0618F4A1E0A0939500409393005093DE
:1004A0009400409191005091920040938F0050939E
:1004B000900042E097C0A09165004A1BA0916600A1
:1004C0005A0B94FD82C093FD80C092FD7CC086FFD4
:1004D00003C0D52EC42E0CC05695479591FD73C010
:1004E0005695479590FD6FC0D52EC42ED694C794CF
:1004F00061FD19C0AC2DAC51AD2DA24008F005C076
:10050000DD2089F4AC2DA85C70F4A0916700A39560
:10051000AA2311F0A0936700AA3008F471C02092BA
:10052000960081606DC0A0916700AA2319F0AA957A
:10053000A0936700A22C5091BA0097FD06C0A0902E
:10054000C800533011F4A090D000AAEFAA0EA22D3B
:10055000A21DCA18DA0A4FB74170533049F4442338
:1005600021F087FD05C0806803C087FF01C08F7739
:10057000442359F0533031F4AFEFC094D094CA1AE9
:10058000DA0A03C040E050E020C0533049F4CC0CFC
:10059000DD1CAAE0CA1AD20818F4A0E0CA2ED22C98
:1005A000AFEFCA16D20418F04FEF50E00EC0A09182
:1005B000AC00CA9E412D000C441F50E008F012C050
:1005C0004FEF50E00FC05695479594FF07C0552355
:1005D00009F04FEFA42FA6954A0F521D4F3F520529
:1005E00008F04FEF40939600816061FF09C0AFE1D2
:1005F000A095A923AB299A2F8F7DBB2009F4806297
:10060000A8E1A093680085FF03C0AAE0A09368005A
:1006100061FD03C085FD01C08F7E85FD03C0A6E09E
:10062000A0936900F894A9B7A160A9BF84FF02C094
:10063000A0E4ABBF3FBE189511E00AC013E008C0AC
:100640001AE006C01EE104C014E602C018EC00C0A7
:1006500005E1BB27BA95F1F70A95D9F71A95C1F7C5
:1006600008952AE338E709C020E33CE806C02AE2FF
:1006700034EB03C025E238EC00C012E0BB27979AA8
:10068000BA95F1F7909ABA95F1F79098BA95F1F773
:100690009798BA95F1F7123009F0919A123009F44F
:1006A000939AB091AD00BA95F1F7123009F0919894
:1006B000123009F49398B7E8BA95F1F71A95F1F664
:1006C000022FB22FBA95F1F70A95D9F73A95A9F604
:1006D000979A0895221B39E0001F3A9509F408956E
:1006E000221F211B18F4210F8894F6CF0894F4CF11
:1006F000622C722CB0E08894B395221F331FE0F770
:10070000379527958894912E802E020B130B10F4A9
:10071000192D082D10F4889401C00894661C771CCC
:10072000BA9571F7172D062D0895322D11232AF44D
:100730003A9500951095031B130BF894029F712CAA
:10074000002D129F912C802C7894780C172D921CE0
:10075000292DB4E06B2E2695179507956A94D9F745
:10076000332321F000951095031B130B089500917E
:10077000B4000430A1F1B0919600B15008F010C05F
:10078000B0916100B093630020927E0020927F00C0
:100790002092800020928100209282006F7B1FC0F7
:1007A0006090B4006064B0916100B093620008E3AF
:1007B00017EC20917A0030917B0036952795B62D65
:1007C000BA9541F036952795B62DBA95BA9511F0A0
:1007D000369527958DDF00937E0010937F00089556
:1007E00000917E00B09162000B1B10917F001209F6
:1007F00028F40038BFEF1B0740F009C00F3712057F
:1008000008F405C00FE710E002C000E81FEF0093F6
:10081000830010938400089500918300B0918000BC
:100820000B0F10918400B09181001B1F20E03091CC
:10083000840033230AF42A95B09182002B1F1AF406
:10084000203F40F00AC02F3008F407C00FEF1FEF21
:100850002FE003C000E010E020EF30916300B09182
:100860009B003B1718F4323030F009C0B09184007F
:10087000BB235AF004C0B0918400BB2332F4009330
:100880008000109381002093820008952091D7006A
:1008900000918300000F10918400111F46DF112387
:1008A0002AF40038BFEF1B0740F009C00F371205CC
:1008B00008F405C00FE710E002C000E81FEF0023B6
:1008C00052F0B0916200B01B0B2F18F0013008F00D
:1008D0000AC001E008C000950F5FB09162000B0FE5
:1008E00008F001C00FEF0093850008952091D80013
:1008F000009181001091820018DF11232AF4013049
:10090000BFEF1B0740F009C00F3F120508F405C0F8
:100910000FEF10E002C001E01FEF112352F0B09181
:100920008500B01B0B2F18F0013008F00AC001E061
:1009300008C000950F5FB09185000B0F08F001C053
:100940000FEF0093630008950FEF677F71FD29C0DB
:1009500072FD09C06860B0917B00BA3020F0B52DFF
:10096000B03408F4677FB091D300BB23D1F0B091CD
:100970007B00BB23B1F00FEF10917B00ABDEF8944E
:10098000B091730072FDB5E00B9F112D002D78948E
:10099000112309F00FEFB0919E000B1710F4009196
:1009A0009E0000939D00089500917A0010917B00B5
:1009B00000541140B0919D0010F4BA9501C0B39558
:1009C00011F0B0939D00089500C008952091B500E6
:1009D000B6B1B6FDFBCF04B115B1B6B1BF77B6B9AC
:1009E000B091AA00B395B093AA00B83060F12092FC
:1009F000AA00B091D200BB2321F1112329F0B091BC
:100A0000AB00BF3F61F009C0B091AB000B1739F0EC
:100A100020F4BB2321F0BA9502C0B395E1F3009115
:100A20009B00B093AB00B03050F400ECB03038F421
:100A300000E8B03020F400E4B03008F400E00093A7
:100A40009B007F7E089510919B00B0E11B0F08F47E
:100A50001FEF10939B00B091B400B43081F000916F
:100A60009B00B0916300B01B10F400916300B09143
:100A70009D000B1708F00B2F502E00936400B091CF
:100A8000AA00B73009F47061089502E3F894B091B8
:100A9000D9000B9F012D000C001F7894B0919B0092
:100AA0000B1710F000919B0000936100009363000E
:100AB000502E0093640000939E00089520927A00C7
:100AC000B0EFB0937B000895F8940CB51DB520915C
:100AD00074007894309175006090760000937500F2
:100AE00010937600031B160971FD03C077FD7DC0CE
:100AF00027C070907700209377002709222311F0F8
:100B00000FEF1FEF8090780090907900309378007D
:100B1000609279000091750010917600081919090A
:100B200020917A0030917B0036952795020F131F94
:100B300010F40FEF1FEF00937A0010937B0029C091
:100B400020917A0030917B003901B4E08B2EB2E025
:100B50009B2E343010F08A949A94383010F08A9496
:100B60009A94769467948A94E1F726193709992024
:100B700021F0169507959A94E1F7200F311F2093E5
:100B80007A0030937B0028F43FEF30937A00309363
:100B90007B00323008F4706871FF02C0B3E00DC012
:100BA000B091C40000917100023838F0B395003A5A
:100BB00008F0B395B63008F0B5E09B2EB4E08B2E6C
:100BC00010917B0000917A0024E0169507952A95F4
:100BD000E1F70819120928F0B02FB250B12FB2096D
:100BE00010F402E010E0980126C020917A003091C4
:100BF0007B0039017694679466946694669426190E
:100C0000320906950695200F321D20937A00309305
:100C10007B00323008F07F7704E0369527953695D3
:100C2000279526952695201B10F0223008F422E007
:100C300089019090C40060FDFECFE0908B00F090A1
:100C40008C006160B9B7B061B9BF380177FD41C0B0
:100C50007694679400938B0010938C00B92DB33079
:100C6000E1F0B0FD04C0060D171D930106C0000F92
:100C7000111F0250120922E030E0B92DB33068F0A4
:100C800020938D0030938E0000938700109388008E
:100C90006092890070928A003AC000938D00109390
:100CA0008E002093870030938800609289007092B4
:100CB0008A0071FF0DC0BFE0B0938D0020928E00BE
:100CC000B093890020928A00B0938B0020928C0010
:100CD0001EC0669400938B00B92DB33091F0B0FD27
:100CE00003C0060D262D03C0000F025022E0B92DCF
:100CF000B33038F020938D00009387006092890014
:100D000006C000938D0020938700609289000091B7
:100D10007C0002FD0350013031F495FD0CC0B2E0BF
:100D2000B06CB7B90BC0023021F4B3E0B06CB7B906
:100D300005C095FDF4CFB4E0B06CB7B90091A20046
:100D4000000F10F4BBE60B270093A20060FDFECF5E
:100D5000B2E0B0936E006160B9B7B061B9BFB72FB0
:100D6000B670D1F020917A0030917B0036952795AE
:100D70003695279571FF02C0B0E43B0FF8940CB58F
:100D80001DB5020F131F1BBD0ABD6160B0E1B8BFE6
:100D9000B9B7B061B9BF78940895606120927D00C1
:100DA00020E067FD20E206C0606120927D0020E225
:100DB00067FD20E001E011E077FD11C0B72FB670AC
:100DC00009F06F7E14E100917B00069509F403950C
:100DD0000F3008F00FE071FF02C004E114E160FD84
:100DE0000FC0B0917D00BB2359F071FF06C0B091D8
:100DF0006E00BA95B0936E0011F4706247C0ABDF1D
:100E0000B0B7B77FB0BFB8B1B0B7B860B0BFB0913E
:100E10007D00B395B0937D00B8B177FD06C0B1E019
:100E200071FDB3E0BA95F1F7B8B1B072B21709F03D
:100E300022C071FF05C00395011708F00A95CFCFB6
:100E400064FD05C00395011708F0B4CFC8CF6F7ECD
:100E5000F8943CB56DB470907A0080907B00370DAB
:100E6000681C6BBC3ABD6160B0E1B8BFB9B7B06196
:100E7000B9BF78949FCFB0916D00B13008F49ACF8C
:100E800064FD98CF0A9509F0AACF7F7D20918D004F
:100E900030918E00F894B0E1B8BF0CB51DB5020FCB
:100EA000131F1BBD0ABDE0908700F09088006160B1
:100EB000B9B7B061B9BF7894B72FB67039F0B091B7
:100EC0006D0072FFB395B0936D0009C075FF07C048
:100ED00067FD05C064FD03C0BF91BF91F1C40895D3
:100EE00000E063FF03C064FF01C001E0F8941091CB
:100EF0007100B7E01B9F212D102D7894200F2695AF
:100F00001795269517952695179510937100183704
:100F100018F4B8E7B093710000917100B0917200BD
:100F20000B1720F0606291989098939860FDFECF27
:100F3000E0908900F0908A006160B9B7B061B9BFF4
:100F40000895B2E095FD0AC0F894B0937C00979A9A
:100F5000949862FF01C0939A7894F4C0F894B09387
:100F60007C00979A959862FF01C0919A7894EAC0A4
:100F7000B3E082FF24C095FD11C002E0F894B09365
:100F80007C00E1E8F0E00093B1009398959A62FF4D
:100F900002C0909A01C097987894D4C002E0F89467
:100FA000B0937C00E1E8F0E00093B1009198949A4E
:100FB00062FF02C0909A01C097987894C3C095FDD3
:100FC0000BC0F894B0937C00EBE6F0E0939862FFDE
:100FD00001C0909A7894B6C0F894B0937C00EBE688
:100FE000F0E0919862FF01C0909A7894ABC0B4E0B1
:100FF00095FD0AC0F894B0937C00949A959862FF8E
:1010000001C0909A78949EC0F894B0937C00959A11
:10101000949862FF01C0909A789494C0B5E082FFE2
:1010200024C095FD11C001E0F894B0937C00E7E77F
:10103000F0E00093B1009098979A62FF02C0919AF5
:1010400001C0949878947EC004E0F894B0937C003A
:10105000EBE8F0E00093B1009098979A62FF02C02D
:10106000939A01C0959878946DC095FD0BC0F89443
:10107000B0937C00E5E6F0E0909862FF01C0919AA1
:10108000789460C0F894B0937C00E1E7F0E0909829
:1010900062FF01C0939A789455C0B6E095FD0AC0EE
:1010A000F894B0937C00959A979862FF01C0919A4A
:1010B000789448C0F894B0937C00949A979862FF13
:1010C00001C0939A78943EC0B1E082FF24C095FDA0
:1010D00011C004E0F894B0937C00EBE8F0E00093DA
:1010E000B1009198949A62FF02C0939A01C09598BA
:1010F000789428C001E0F894B0937C00E7E7F0E032
:101100000093B1009398959A62FF02C0919A01C032
:101110009498789417C095FD0BC0F894B0937C0018
:10112000E1E7F0E0919862FF01C0939A78940AC0D9
:10113000F894B0937C00E5E6F0E0939862FF01C07C
:10114000919A78946F7D089524E630E0F901209219
:10115000B100919890989398949A979A959A6B7FEA
:101160000895A2EBB0E009E00D9309E00D9304E0CF
:101170000D930FEF0D9303E00D930FEF0D930AE026
:101180000D9303E00D9301E00D9301E00D93AEEBA1
:10119000B0E001E00D930FEF0D930D930D930D93C0
:1011A0000D9303E00D930FEF0D930FEF0D930D9340
:1011B00005E20D9300ED0D9308E20D9300E50D930C
:1011C00004E00D930FEF0D9302E00D9300E00D93FB
:1011D0000AE70D930FEF0D9300E00D9301E00D93DF
:1011E00000E00D9303E00D9300E00D93089520912E
:1011F000B9008B7F233009F48460B091BA00B3301A
:1012000019F09F7DB1FD90629F7BB091BB00B1FD55
:101210009064223011F0886001C0877F08950A959C
:10122000E00FF21DB4910895ECE1F0E00091B200FE
:10123000F6DFB093D700ECE1F0E00091B300EFDF10
:10124000B093D800EAE2F0E00091B800E8DFB09394
:10125000D9000091B800023008F402E00093730056
:10126000B091CE000FEFB23009F400EAB33009F4C8
:1012700002E800937200E8E3F0E00091D500CFDFD0
:10128000B093A000089508952091C8003091C9003E
:10129000B091BA00B33009F43E5097FF02C020E08D
:1012A0003FEFB32FB21B6B2EB25810F4B2E86B2E87
:1012B00000E00395609EB12DBD57D8F30093AC00BC
:1012C00008959068E1DFBED920E030E0B0E16B2EF8
:1012D000B5D9B09196002B0F321D6A94C9F7B4E0CE
:1012E00036952795BA95E1F7822E9F77CDDF089541
:1012F000F894E3E0F0E0B9E0B7BFB491B078C1F39F
:10130000F894A895B1B5B861B1BDB0E0B1BDB4E095
:10131000BEBFBFE5BDBF18DFB0E0B8BBB0E1B7BB33
:10132000B0E0B5BBB0E0B4BBB0EBB2BBBBEBB1BBA4
:101330002224A0E0B0E02D92AA31E9F7A0E6B0E0C7
:101340000FEF2D920A95E9F7B1E0B093A20009DF03
:10135000F3D2B7E0B06CB7B9B6B1B460B068B6B9A3
:101360000091CA000093AD00B1E0B0936A00F89418
:101370006DD977D967D978D965D979D963D9F894EE
:101380000AEF1AEFA0B396FFA095A2FF1FC01A950F
:10139000C9F70A95B1F7E0E0FCE1B591B43E39F444
:1013A000B591B03E21F4B591BF3F09F40CC0E0E027
:1013B000F395F395B591B83F49F4B591B43931F44B
:1013C000B591BA3A19F4EE27F695099410DF2CDF9F
:1013D0005ADF5ADF0091CA000093AD00B5DEB2E0DB
:1013E000B3BFB2E0BEBDB2E0B5BDB1E5B8BFB9BFF5
:1013F000B0B7B77FB0BFB8B1B0B7B860B0BF1CD995
:101400007894E2DA20927000B3E096FFB2E0B5BFC4
:10141000B0E4BBBFBB27B064BABF8D7F17D9626091
:1014200033E02CE0B0919500BB2321F42CE03A95F9
:1014300009F4A5CF07D980FFA2CF8E7FB091960087
:10144000B23078F3B92FBF710091980000939700E4
:10145000B0939800B01729F72A9521F76D7FB3E074
:1014600096FFB2E0B5BFBB27B064BABF8D7FB09125
:10147000D400BB2321F48062B92FB0709B2F8F7BE7
:1014800020926700E1D885FF05C0B0916700BA30AF
:1014900008F08064D3D802E085FF01C000E0B0917D
:1014A0009600B017B8F3F894DCD8DBD8DAD8789483
:1014B000CDD820928600B091BA00B33009F473C041
:1014C000BDD8B091BE00B13008F46DC0B0916A00D3
:1014D000B13008F468C085FD18C0B0919600BF3FD8
:1014E00008F461C0F894C6D87894AED8B09196004C
:1014F000B130C0F7F894B5D8A3D8B3D87894A4D8AD
:10150000B0919600BF3FB0F3D8C2B3E09B2E906875
:10151000F894BADE789498D8F8949F77B5DE8090E6
:101520009600B0919600BF37789408F444C084D8F0
:10153000F894A0D878949A9451F7C3DEB82DB0935C
:10154000C90084D8F89425D28BD27894BAE09B2E27
:101550009068F89499DE789477D8F8949F7794DE21
:1015600080909600B0919600BF37789478F764D851
:10157000F89477D865D875D878949A9449F7A1DE0D
:10158000B82DBB5FB093C80061D8F89402D277D26F
:1015900078945AD8F89478DE7894B0919600BF3F4A
:1015A00008F499CF8AC200919600B09186000B177B
:1015B00010F00093860048D801E0B091BA00B35013
:1015C00009F405E0B0919600B01708F074CFF894D4
:1015D00051D850D84FD8789439D820926A002092A8
:1015E0006B0020926C00B0916B00B395B0936B00D0
:1015F000BF3F71F5B0916C00B395B0936C00B091A2
:10160000CC0009E1BA9559F002E3BA9541F00DE733
:10161000BA9529F00AEFBA9511F020926C00B091BA
:101620006C00B017A8F090DD07D8B0916C00BA95A7
:10163000B0936C0020926B00B091CB00B093AD00E2
:10164000F89418D87894B091CA00B093AD00FCD744
:10165000F7D7B0916800BB2319F485FF01C08FCE86
:1016600001E085FD01C006E0B0919600B01708F4D6
:10167000BACFB091BA00B35009F0E6D7B091680084
:10168000BB2309F47CCEF8945FDD209261002092A8
:10169000620020926300522C209264002092A100EC
:1016A0007894B091B700BB0FB0939F0020927E005A
:1016B00020927F0020928000209281002092820060
:1016C0002092AA0060E070E020927100B8E0B09330
:1016D000AA007061B1D7B7E074FDB7E0B06CB7B9DC
:1016E000B6B1B068B064B6B9B6B1B6FDFDCF04B15D
:1016F00015B1B6B1BF77B6B9112309F00FEF00935A
:10170000AB0064D9B8E0B093AA00706170DDF894C2
:10171000BFEFB0939B00B9D9B0916100B0939B002B
:10172000B0939C00B0939D007894B1E0B0936100B9
:10173000B09363005B2EB0936400B093A400B091AB
:101740009A00B093A300B091BA00B33019F49F7D12
:1017500087FD90627160726020926D009EDCB4DC47
:10176000ADD9B2D9ABD9B0D9A9D91EDB00D8B8DB75
:10177000E8DBAAD912DB66FD33D877FFE5D877FD21
:1017800013D9AEDBF5DBA0D90FDB66FD45D8A8DBAE
:101790002EDC9AD902DB66FD79D8A2DB3FDC94D936
:1017A00003DB66FDA3D89CDB78DC8ED9F6DAB7E0E4
:1017B00074FDB7E0B06CB7B9B6B1B068B064B6B993
:1017C0008FDB82DC81D902D971FF24C0B0919E00E9
:1017D000B0939B00B0939C00B0919A00B093A3008B
:1017E000B1E0B093A40018E12CE0B0916D00B11706
:1017F00058F07D7F746020936F00B0919E00B0938D
:101800009B00B0939D0006C0B0919600B13008F0E7
:10181000ACCF60C072FF11C067FD0FC0B0916F0008
:10182000BA9519F47B7F7860A0CFB0936F00B09128
:101830009600B13008F099CF4DC020927000B09161
:1018400099000AEF1091D600112309F003E0B017B8
:1018500008F040C085FF04C0B0916800BB23D1F1FF
:10186000B091BA00B33081F495FD03C087FD04C088
:101870000BC087FF01C008C067FD06C06068B0915B
:101880009E00B0939B0086CF00EF67FF05C0B0912C
:101890009E00B0939B0000E2B0917B00B01708F46B
:1018A00064CF67FF17C06F779F7D87FD906274607C
:1018B000B2E1B0936F00B0919E00B0939B0055CF02
:1018C000B0917000B395B0937000B0919600BB23B7
:1018D00009F002C020927000F89436DC8090B900C4
:1018E000B2E0B093B90083DC8092B900209261002D
:1018F0002092620020926300522C20926400209279
:101900009F0060E070E078949FD61EDC0091D600C6
:10191000002319F0919A909A939AB7E0B06CB7B9F6
:10192000B6B1B460B068B6B985FF05C0B0917000BB
:10193000B43008F024CD53CEEDE0F0E023D00535EF
:1019400009F01BC0EEE0F0E01DD00A3A09F015C026
:101950003AE0A2EBB0E0E3E0F0E014D00D93319672
:101960003A95D9F739E1AEEBB0E0EFE0F0E00AD01C
:101970000D9331963A95D9F702C0F3DB0AD0E8E22D
:10198000F0E00895E199FECFEEBBFFBBE09A0DB306
:1019900008951ED03AE0A2EBB0E0E3E0F0E00D9154
:1019A0000FD031963A95D9F739E1AEEBB0E0EFE0E0
:1019B000F0E00D9105D031963A95D9F712D00895FF
:1019C000E199FECF0DBBEEBBFFBBE29AE19A089511
:1019D000EDE0F0E00FEFF4DFEEE0F0E00FEFF0DF2E
:1019E0000895EDE0F0E005E5EBDFEEE0F0E00AEA77
:1019F000E7DF08953091AE000091AF00313011F46F
:101A00000093B200323011F40093B300333011F47C
:101A10000093B400343011F40093B600353011F463
:101A20000093B800363011F40093C400373011F43D
:101A30000093B900383011F40093D500393011F417
:101A40000093CE003A3011F40093BA003B3011F409
:101A50000093BB00089525E0F9D52A95E9F708958C
:101A600000D602D604D606D6EBD5FBD5FDD5FFD5DC
:101A700001D6E6D5F6D5F8D5FAD5FCD50895FAD530
:101A8000F6D5F2D5EED5DCD5F5D5F1D5EDD5E9D540
:101A9000D7D5F0D5ECD5E8D5E4D508958090AE0043
:101AA0009090AF00DED5DDD5DCD5CAD58A94D1F7CC
:101AB000E1D5C6D59A94E1F70895F894D1DF7894EA
:101AC000CADFC9DFB1E0B093AE00B1E0B093AF00C0
:101AD0002092B000F894E2DF7894B5E06B2E70901D
:101AE0009600B4D5B09196007B16C9F7B13018F0C6
:101AF000BF3F40F107C07EDFF8944BDFB1DFB8E0B5
:101B0000B1BDA9DF6A9459F7B091B000B395B09315
:101B1000B000B33008F4DECF9EDFB091AF00B395D4
:101B2000B093AF00F894B091AE00BA95EEE3F0E058
:101B3000EB0FF21D049178940395B091AF00B017AC
:101B400008F4C6CF88DF87DFB091AE00B395B093BD
:101B5000AE00B091AE00BC3008F4B7CF02DBF89411
:0A1B600018DFB8E0B1BD77DFC3CB9A
:00000001FF
